:020000020000FC
:020000001EC020
:0200140005C223
:0200180091C194
:10003C00EDC101E20EBF0FEF0DBF07E104B908E0FF
:10004C0005B901E00DBD00E50CBD289A2C980F9A5E
:10005C00179A0CE000936A0000E20DBB0AEAA02E8E
:10006C000BEBB02ED2E0C0E022275524992788272D
:10007C007727A89500E004BF0EE10093600006E02E
:10008C00009360000BEA009364000FE3009365009B
:10009C0000E900BF00E20093B60005E00093B10058
:1000AC000091B6000F71E1F700270093170001E0F3
:1000BC0000937000689A7498B3D140E8FED0A8D031
:1000CC0003EC2898F4D00027F2D0289A00EE289858
:1000DC00EED000EFECD0289A01EE2898E8D00AEA8E
:1000EC00E6D0289A02EE2898E2D00DECE0D0289ABF
:1000FC0003EE2898DCD00BEADAD0289A08EC289882
:10010C00D6D006E3D4D0289A05EC2898D0D000E8B5
:10011C00CED0289A0CEE2898CAD008E3C8D0289ADA
:10012C000EEE2898C4D007E0C2D0289A0DEE28987D
:10013C00BED000E8BCD0289A0FE82898B8D0289AEE
:10014C000EEC2898B4D008E0B2D0289A00270CBB4B
:10015C0078942C9A40E8B1D0F894A8950EE10093CD
:10016C0060000EE000936000789483D1A8D12C98A5
:10017C0048E2A3D053D07DD05C3028F0C0E05FE0E3
:10018C0017D222E002C052D220E000000000000092
:10019C00203421F1203899F0243009F0F6CFAFEF5C
:1001AC000000000000000000000000000000000043
:1001BC00000000000000243041F7AA9589F75C305C
:1001CC0068F469927992399249920992199229921A
:1001DC0099935395D33010F0D2E0C0E028D02C9AEC
:1001EC0007E003BF6CE3F894A89504B7077F04BF3E
:1001FC000EE10093600006E000936000789488950F
:10020C000000000000006A95D1F7002703BFA4CFBF
:10021C0002EC28984CD008E04AD0289A01E828989B
:10022C0046D000E044D0289A0830C1F7089502EC7B
:10023C0028983DD003E03BD0289A00000000000035
:10024C00000001E8289833D000E031D0289A08301B
:10025C0071F7089502EC28982AD009E028D0289A42
:10026C0001E8289824D000E022D0289A0930C1F760
:10027C00089502EC28981BD009E119D0289A01E8BE
:10028C00289815D000E013D0289A0931C1F70895A9
:10029C0002EC28980CD006E10AD0289A01E828989C
:1002AC0006D000E004D0289A0631C1F708950EBD9F
:1002BC000DB507FFFDCF0EB508950000000000003E
:1002CC00000000000000000000004A95B1F70895FE
:1002DC00243051F500E22898EADF00E0E8DF0B302B
:1002EC00F9F400E0E4DF00E0E2DF00E0E0DF0630FC
:1002FC00B9F400E0DCDF00E0DADF00E0D8DF00E09A
:10030C00D6DF00E0D4DFB02E00E0D1DFA02E289A9B
:10031C00C5DFA0DFAEDF8AD120E10F910FBF1895AA
:10032C00289A0F910FBF189520E40F910FBF1895C5
:10033C000FB70F930FE82898BADF289A01E828988E
:10034C00B6DF00E0B4DF289A063111F2013101F278
:10035C000F31A1F3023191F302E82898A8DF00E0F5
:10036C00A6DF289A007E0036A0F0203041F0203124
:10037C0061F0203249F020E40F910FBF189518D18D
:10038C0022E00F910FBF1895C52D20E80F910FBFDC
:10039C001895203039F02230B9F0203259F0203144
:1003AC0009F0C2CFC03031F05C2E1ED120E20F918B
:1003BC000FBF1895552720E40F910FBF189536D114
:1003CC0020E00F910FBF189545DF62DF24E00F91FD
:1003DC000FBF18952C9A00002C9800E6289867DF20
:1003EC000BE065DF00E463DF08E861DF00E05FDF5E
:1003FC000DEC5DDF0BEA5BDF0FEF59DF0FEF57DF23
:10040C0000EF55DF0AEA53DF289A08950000000038
:10041C0000001895000000000000EC9800001895F2
:10042C00B1D09ED0709A7098709A7098709A70989B
:10043C00709A7098709A70986C98709A7098709A6C
:10044C0070986C9A709A709895D06C9A709A709803
:10045C00709A7098709A7098709A7098709A709848
:10046C00709A7098709A70986C98709A709882D0F4
:10047C00089576D0709A7098709A7098709A709857
:10048C00709A7098709A7098709A70986C98709A1C
:10049C007098709A70986ED0EC9A07E003BF0000C9
:1004AC00000000008895000000000000002703BF3A
:1004BC0035D02FD0002E32D029D0102E089550D008
:1004CC00709A7098709A7098709A7098709A7098D8
:1004DC00709A70986C98709A70986C9A709A7098D0
:1004EC006C98709A709846D0EC9A07E003BF0000A5
:1004FC00000000008895000000000000002703BFEA
:10050C000DD007D00BD002D0202E0895709A709881
:10051C0008956C9A709A70986C9808950027709A48
:10052C00649900687098709A649900647098709AD5
:10053C00649900627098709A649900617098709ACE
:10054C00649908607098709A649904607098709AB5
:10055C00649902607098709A64990160709808951B
:10056C006C987098709A6C9A7098709A6C98709845
:10057C006C9A08956C986499FECF709A7098649BED
:10058C00FECF08956C98709A7098709A7098709AC3
:10059C007098709A7098709A7098709A7098709A07
:1005AC007098709A7098709A7098709A7098089564
:1005BC002C9A00002C9800E6289879DE0BE077DE68
:1005CC0000E475DE08E873DE01E071DE0DEC6FDE31
:1005DC000BEA6DDE0FEF6BDE0FEF69DE00EF67DE0F
:1005EC000AEA65DE289A08952C9A00002C9800E6F9
:1005FC0028985DDE1C2F0BE0010F59DE01E657DE5B
:10060C0008E855DE04E053DE0DEC51DE0BEA4FDE5C
:10061C000B2D4DDE0A2D4BDE00EF49DE0AEA47DEDC
:10062C000A9145DEC030E1F7289A08952C9A000013
:10063C002C9800E628983BDE03E139DE01E637DE34
:10064C0008E835DE02E033DE0DEC31DE0BEA2FDE9E
:10065C000B2D2DDE0A2D2BDE00EF29DE0AEA27DE1C
:10066C00092F25DE022D23DE012D21DE002D1FDEBC
:10067C00042D1DDE032D1BDE072D19DE062D17DEC6
:04068C00289A08950B
:00000001FF
